:020000040000FA
:020000001C28BA
:040002000034003492
:080008000528F0000308F100D7
:1000100083010C180E280B19132817288E018F0145
:10002000B4140C1017280B118715871117287108A5
:100030008300F00E700E090083160F178F160F162F
:10004000FF30920000309F0007110514851405153C
:10005000851601308C0007308100031788010814D1
:1000600088140815081689018312031340308B0089
:10007000303090003C309700043092000A30A900E4
:10008000C10100304421A300950001304421A100AA
:1000900002304421AA0003304421AB000430442143
:1000A000AC0005304421AD0006304421AE004D21A6
:1000B000E5208E018F018B171014B4018930302197
:1000C000B300B418842091303021A0008130302159
:1000D000B10085303021B2003102031C3208031810
:1000E0003108A20020082102031C2D212008220231
:1000F00003187F281508003C031C95035E2815088B
:1001000023020318950A6128023063213308A921CC
:1001100026086621270866212E30662128086621D8
:1001200056306621203066214330662143306621F7
:100130003D3066210310B4122A08BA006430B500BD
:100140002008DD21F2213D083E18B416A921260819
:1001500066212E3066212708662128086621423054
:100160006321B4122B08BA006430B5003108DD21D8
:10017000F2213D083E18B416A921260866212E302A
:100180006621270866212808662141306621203033
:10019000662120306621203066212D306621B41280
:1001A0002C08BA006430B5003208DD21F2213D0888
:1001B0003E18B416A921260866212E30662127088C
:1001C000662128086621B4100800003063215630EB
:1001D00066213D30662130306621303066212E3078
:1001E000662130306621563066212030662143304A
:1001F0006621433066213D306621303066212E3045
:100200006621303066213030662141306621403031
:100210006321203066212B306621303066212E305C
:100220006621303066213030662141306621203031
:10023000662120306621203066212D306621303045
:1002400066212E3066213030662130306621413003
:1002500066210800B418842008002108A0000800C6
:100260009F000000000000000000000000000000EF
:1002700000000000000000000000000000009F14CB
:100280009F1840291E08080003178D0083168C1341
:100290000C1483120C080313080083160313861230
:1002A00006128611061187120712831203130A22FF
:1002B00028308721283087210C30872160210800D1
:1002C000013087210800803887210800A4001E2201
:1002D000071687168612061286110611A41B8616AB
:1002E000241B0616A41A8615241A061587128716CB
:1002F000A40E8612061286110611A41B8616241B54
:100300000616A41A8615241A061587120800A400DA
:100310001422071287168612061286110611A41BD4
:100320008616241B0616A41A8615241A061587128B
:100330008716A40E8612061286110611A41B8616B5
:10034000241B0616A41A8615241A061587121422D1
:100350000800A5000030A600A700A8006430250210
:10036000031CB529A500A60AAE290A302502031CE4
:10037000BC29A500A70AB5292508A807B41ED729B6
:100380002808063EA800A50029082502031CCA2942
:10039000A70AA8002708053EA500A70029082502EE
:1003A000031CD429A60AA7002608023EA600303066
:1003B000A607A707A807B41208000310B801B901DF
:1003C000B600B701B50C031CEB293708B90736088E
:1003D000B8070318B90A0310B60DB70DB508031D09
:1003E000E22908003908BC00C0003808BB00BF0083
:1003F000BE01BD014008A5003A083F02031CA50349
:10040000A51B092ABF002508C000BD0A0319BE0AA2
:10041000FA2908007730AF00B000AF0B0D2A773013
:10042000AF00B00B0D2A08002D08AF00B000AF0BD5
:10043000172A0A30AF00B00B172A08002E08AF00A9
:06044000AF0B202A0800AA
:02400E0084200C
:02401000FF3E71
:00000001FF
